:1000000031C04BC03DC349C048C047C046C045C0D1
:1000100044C043C042C041C040C03FC03EC00902CE
:10002000190001010080640904000001FF000000C4
:100030000705810308000A12011001000000088171
:10004000179F0C04010002000116035500530042E3
:1000500000740069006E00790053005000490004EC
:100060000309040011241FBECFE5D1E0DEBFCDBFE0
:1000700010E0A0E6B0E0EEEAF9E002C005900D92D3
:10008000A436B107D9F720E0A4E6B0E001C01D9284
:10009000AB3AB207E1F752D488C4B2CF9C01DC017D
:1000A0001496F901E0812F5F3F4F48E050E090E85F
:1000B00080E0FE2FF92309F0C09AF09160000F2E26
:1000C00000C00000000000000A94D1F7C29AF0912D
:1000D00060000F2E00C00000000000000A94D1F75D
:1000E000880FB1998F5FC098C29896954150510979
:1000F00001F7FB018193A217B30709F40895BF012B
:10010000D0CF80916F00909170009C012F5F3F4F86
:100110003093700020936F0020916C0027FF11C076
:10012000880F991F20936800292F26952093690036
:100130009695879580936A0064E670E088E690E083
:10014000ADCF80FFEFCF2860EDCFEF92FF921F93EE
:10015000CF93DF93162FEC017C01E60EF11CCE1538
:10016000DF0539F4812FDF91CF911F91FF90EF9040
:100170000895C7DF809167008993F1CFDF92EF92F6
:10018000FF920F931F93CF93DF93EC018C01060F27
:10019000111D30E6D32EC017D10749F481E0DF915D
:1001A000CF911F910F91FF90EF90DF90089589916B
:1001B00080936B00A6DF809168008D258093680096
:1001C000F12CE12C80916D0090916E00E816F906FB
:1001D00010F764E670E088E690E060DF90916700D9
:1001E00080916B00891308C090917200981721F0DC
:1001F000909171009813CFCF8091600090E025E03E
:10020000880F991F2A95E1F7E80EF91EDBCFCF93EF
:10021000DF93EC018981811108C0D0939000C093D5
:100220008F0088E0DF91CF910895EC81F0E081307C
:1002300039F490819883D0939000C0938F00F2CFCF
:100240009A81823019F4908380E0ECCF492F477077
:1002500021E030E001C0220F4A95EAF7833029F40B
:100260002095808128232083EFCF843019F480816A
:10027000282BF9CF853051F490936000B99887B35B
:10028000856287BB88B3887D88BBDECF863019F452
:1002900080E287BBF9CF873051F4BE01CE010296D0
:1002A000FDDED0939000C0938F0084E0BBCF8830F8
:1002B00031F4909372008B8180937100C5CF2C81B3
:1002C0003D813093700020936F00893029F480E2E3
:1002D00080936C008FEFA6CF8B3011F480EAF8CFBB
:1002E0002A813B8130936E0020936D008A3011F497
:1002F00080E4EECF8C3009F0A7CF80ECE9CFDF921D
:10030000EF92FF920F931F93CF93DF9388E0E82E35
:10031000F12CC0E0D0E8DD2EDC0ED1BE9ED18C01E8
:10032000043389E018070CF4CD2DD69581E0E81A46
:10033000F10889F78FEF8C0F81BFEC2EF12C8FEF36
:10034000E81AF80A81B78E151F0469F064F0C1BF7E
:1003500061B790E080E0DF91CF911F910F91FF9006
:10036000EF90DF9014C379D18453994097FF03C075
:100370009195819591098017910714F4C1B78C016B
:1003800081B78F5F81BFDECFCF93C62F20918000D2
:1003900024FF1BC02091810038E82327209381008F
:1003A000E2E8F0E09C01D9012F5F3F4F9C919193CF
:1003B0009C2F921B980FB9F76C2F82E890E049D1DF
:1003C000CC5FC0938000CF9108952AE520938000F0
:1003D000E7CFCF93DF9360919100635067FD90C0AA
:1003E00080918E00CCE0D0E0C81BD109CB56DF4F06
:1003F00080918D008D3209F0CCC0683009F07EC04C
:1004000083EC809375008AE58093620010927400FB
:100410008881807671F0CE01FADE8F3F09F466C0E4
:100420009F81911169C09E81981708F065C0892F3E
:1004300063C02A8110927E00998191110AC01092A6
:100440007F002EE730E082E03093900020938F0011
:10045000E7CF953029F4209392002EE730E0F4CFD7
:10046000963071F59B81913059F487E390E0909339
:10047000900080938F0082E190E490937400D0CF3D
:10048000923041F48EE190E09093900080938F0041
:1004900089E1F2CF933081F7211108C08FE590E018
:1004A0009093900080938F0084E0E6CF223021F774
:1004B00089E490E09093900080938F0086E1DCCFF8
:1004C000983069F0993019F420939400C6CF9A308F
:1004D00051F09B3011F69BE490938100BECF24E94C
:1004E00030E081E0B1CF2EE730E0FBCF988197FD7F
:1004F0008E8190E890937400809361001092910037
:100500008091620084FF2DC0809161008F3F49F18E
:10051000C82F893008F0C8E0982F9C1B9093610089
:100520009091750028E8922790937500882361F0D8
:100530002091740027FF3FC06C2F86E790E005DE16
:10054000C82F893008F060C06C2F86E790E081D01A
:1005500084E08C0FC83019F09FEF90936100809376
:10056000620084E196B3987131F48150D9F710920A
:10057000920010928C00C1E08111C0E09091730054
:10058000C91721F08111BBDEC0937300DF91CF91B9
:1005900008958091740087FFB1CFCE01EFDD8F3FCA
:1005A00021F48EE180936200A9CF882309F4A6CFBD
:1005B00010926100A3CF80918F009091900026FF50
:1005C00019C0FC0126E730E04C2F480F5491D901A7
:1005D0005C932F5F3F4F31964E13F8CF2FEF2C0FC8
:1005E00030E02F5F3F4F820F931F909390008093D6
:1005F0008F00AACFA6E7B0E0FC012C2F280F319185
:100600003D932E13FCCFEACF8FEF809361008EE1F4
:10061000A6CFAC9A8BB780628BBFE0E8F0E08BE4AA
:1006200081838AE580830895A82FB92F80E090E028
:1006300041E050EA609530E009C02D9182279795FE
:10064000879510F084279527305EC8F36F5FA8F375
:100650000895EADF8D939D930895A6E08827992752
:10066000AA9569F00197E1F3B399FCCFB39BFECF54
:1006700081E09927A6B3019611F0A871D9F70895E2
:10068000CF93CFB7CF93C395B39BE9F7B39B0BC081
:10069000B39B09C0B39B07C0B39B05C0B39B03C00A
:1006A000B39B01C0D5C00F92DF93C0918E00DD27B0
:1006B000CB56DF4F012EB39B03C0DF910F90E6CFE7
:1006C0002F930F931F934F932FEF4F6F06B303FB9F
:1006D00020F95F933F9350E03BE065C016B30126DD
:1006E000502953FDC89556B3012703FB25F92F73F5
:1006F00006B3B1F05027102713FB26F906B22230BB
:10070000F0F000C016B3012703FB27F9012650299A
:1007100006B22430E8F54F77206816B30000F6CF14
:1007200050274F7D206206B2102F000000C006B394
:1007300000265029102713FB26F906B2E2CF4F7B83
:1007400006B3206400C0DACF01265029187106B222
:1007500069F14E7F2160012F16B328C00026502971
:100760004D7F06B22260102F29C0012650294B7FF1
:1007700006B22460012F2DC016B301265029477FF1
:100780002860000006B22EC04F7E06B3206130C044
:10079000422706B3499300265029102706B24FEF8F
:1007A00013FB20F9297F16B379F2187159F101264C
:1007B000502906B2012703FB21F9237F06B371F20A
:1007C000002650293150D0F006B2102713FB22F931
:1007D000277E16B351F201265029012703FB06B2EA
:1007E00023F92F7C49F2000006B3102713FB24F9EC
:1007F0000026502906B22F7939F270CF10E21ABFC5
:10080000002719C03B503195C31BD04010E21ABFDE
:100810000881033C09F10B34F9F020918C00198117
:10082000110F1213EDCF4A81441F093651F10D32D9
:1008300011F0013E29F7009393003F915F914F9192
:100840001F910F912F91DF910F90CAB7C5FD1BCF5C
:10085000CF91CFBFCF91189520919300222369F3B8
:1008600010919100112379F534307AF13093910091
:1008700020938D0010918E003BE0311B30938E0051
:1008800024C0009191000130F4F40AE54F7049F45E
:100890003091620034FD1AC000936200C5E7D0E0D9
:1008A00019C03091800034FD11C000938000C1E870
:1008B000D0E010C0052710E000C021C0052710E0DF
:1008C000C89508BB14C03AE501C032ED032EC0E064
:1008D000D0E032E017B31861C39A08B317BB58E1F0
:1008E00020E84FEF20FF052708BB279517951C3FF1
:1008F00028F700004552B0F720FF0527279508BBD1
:1009000017951C3FB8F629913A9561F7077E10912B
:100910009200110F08BBC250D04011F010938C0010
:1009200010E21ABF086017B3177E402F477E54E0CD
:100930005A95F1F708BB17BB48BB7FCF80E287BB56
:1009400088BB90E080E01BD08F3F09F081BFBB9A4D
:1009500084E1E2EBF1EF3197F1F700C00000815044
:10096000C1F7BB9888E19EE00FB6F894A89581BDC9
:100970000FBE91BD4EDE7894A8952BDDFDCFE19999
:10098000FECF1FBA8EBBE09A99278DB30895262F0C
:10099000E199FECF1CBA1FBA8EBB2DBB0FB6F894DF
:0E09A000E29AE19A0FBE01960895F894FFCFF7
:0409AE0032FF5A00BA
:00000001FF
